:1000000093086008730000009308100817050000AB
:100010001305A51D970500009385251E730000009C
:1000200093081008170500001305851C97050000AC
:100030009385C51D73000000930810081705000084
:100040001305551B970500009385851C7300000060
:10005000930850087300000065DD930870081705C9
:10006000000013058516C145170600001306E616A5
:10007000C14673000000170500001305051597051C
:10008000000093856519292A61D593081008170582
:10009000000013058515970500009385451673002C
:1000A00000000545F520930810081705000013050A
:1000B0002514970500009385351573000000094548
:1000C000C1289308100817050000130505129705AD
:1000D000000093853513730000000D4555289308E3
:1000E0001008170500001305F5109705000093850B
:1000F0005512730000001545612893081008170574
:1001000000001305E50E9705000093852510730088
:1001100000002945B528930850087300000015CD4C
:1001200093087008170500001305250AC145170636
:1001300000001306860AC146730000001705000080
:100140001305A508970500009385050D912861D535
:1001500093086008730000006DBF9308100817052E
:10016000000013053509970500009385650A7300A3
:1001700000000945312893081008170500001305F1
:10018000C506970500009385450773000000ADBDC7
:10019000F32210C01695F32210C0E3EEA2FE828077
:1001A000814233035500B383550003030300838367
:1001B00003008502631773008143E31473FE054552
:1001C00082800145828020202020202020202020A5
:1001D000202020202020202020202020202020201F
:1001E0002020202020206C696768740062656C6C98
:1001F0000067617465004F46460059454C4C4F57A7
:1002000000524544006F6E006F66660075700064B2
:0C0210006F776E00646574656374000015
:00000001FF
